:107E0000112494B714BE892F8D7011F0892FDED004
:107E100085E08093810082E08093C00088E18093B8
:107E2000C10086E08093C2008CE08093C4008EE0A5
:107E3000B7D0559A86E023EC3FEF91E03093850070
:107E40002093840096BBB09BFECF4D9AA89581509D
:107E5000A9F7EE24FF24B3E0AB2EBB24B394A5E036
:107E6000DA2EF1E1CF2E90D0813471F48DD0082F2D
:107E70009DD0023811F482E005C0013811F486E08B
:107E800001C083E079D075C0823411F484E103C06D
:107E9000853419F485E092D06CC0853579F474D0BE
:107EA000E82EFF2471D0082F10E0102F00270E2994
:107EB0001F29000F111F7AD078015BC0863521F48D
:107EC00084E07CD080E0DECF843609F035C05CD021
:107ED0005BD0182F59D0082FC0E0D1E055D089933E
:107EE0001C17E1F763D0053409F4FFCFF701A7BEF3
:107EF000E89507B600FCFDCFA701A0E0B1E02C910A
:107F000030E011968C91119790E0982F8827822B62
:107F1000932B1296FA010C01B7BEE89511244E5F1F
:107F20005F4F1A1761F7F701D7BEE89507B600FC57
:107F3000FDCFC7BEE8951DC0843769F425D024D095
:107F4000082F22D033D0E701FE018591EF0114D034
:107F50000150D1F70EC0853739F428D08EE10CD00E
:107F600085E90AD08FE08ECF813511F488E018D0F2
:107F70001DD080E101D077CF982F8091C00085FF80
:107F8000FCCF9093C60008958091C00087FFFCCF7E
:107F90008091C00084FD01C0A8958091C60008951D
:107FA000E0E6F0E098E1908380830895EDDF803291
:107FB00019F088E0F5DFFFCF84E1DECF1F93182FA3
:107FC000E3DF1150E9F7F2DF1F910895282E80E0DA
:087FD000E7DFEE27FF2709940B
:027FFE00020679
:0400000300007E007B
:00000001FF
